:10000000B728FF3FFF3FFF3FA53003138312DA00FD
:10001000DA0B082800000000080003138312A50172
:10002000210884000008D3000130D1002208D2004A
:100030005108D000520803192128D00D5010FF3F5D
:100040001B285308D0055008D100520803192C284A
:10005000D10CD113FF3F262851082406031D5A282E
:100060002308003C0318382804200420A303302868
:10007000210884000008D3000130D1002208D200FA
:100080005108D000520803194928D00D5010FF3FE5
:1000900043285308D0055008D100520803195428AA
:1000A000D10CD113FF3F4E2851082406031D5A28B6
:1000B000FF30A5002508D000080003138312851621
:1000C0004130DB00FF30DA00DB0B67286A28DA0BEF
:1000D00067286428C330DA00DA0B6C2800000515A5
:1000E0004130DB00FF30DA00DB0B77287A28DA0BAF
:1000F00077287428C330DA00DA0B7C2800008514D6
:100100000730DB00FF30DA00DB0B87288A28DA0BA8
:10011000872884287830DA00DA0B8C280000000069
:100120000514080003138312051085104130DB000D
:10013000FF30DA00DB0B9D28A028DA0B9D289A28D7
:10014000C330DA00DA0BA228000005114130DB00D1
:10015000FF30DA00DB0BAD28B028DA0BAD28AA2877
:10016000C330DA00DA0BB22800008512080007302D
:1001700003138312990083169F01183085001830ED
:10018000831285000530A1000430A2006430A30072
:10019000A4010D205008FF3A031DDB285D2000302C
:1001A000051A0130D1005108003A031DD92800007A
:1001B000CF289220C2280530A1000330A2000530CC
:1001C000A300A4010D205008FF3A031D17295D204C
:1001D000003085190130D1005108003A031DF22882
:1001E0000000E828A001A0012008FF3C031C1529FD
:1001F0000430DB00FF30DA00DB0BFF280229DA0BCA
:10020000FF28FC28E230DA00DA0B042900308519D7
:100210000130D1005108003A031D0F29E8282008B9
:10022000FF3A03191529A00AF4289220DB28C228D6
:100230001829FF3FFF3FFF3FFF3FFF3FFF3FFF3FCB
:02400E00543F1D
:00000001FF
